:10000000922864001120031801281C2008308F005A
:100010001D2011208E0C0C288F0B08281D200E0887
:100020000800220884002008841780048413000537
:100030001F192006FF3E08001F171F0D06398C00F0
:100040002B208D008C0A2B201F1F71281F138C0062
:1000500002308820712800308A000C0882070134A1
:1000600075340334153400343C340C34D9348F00E7
:100070002208840020095E2084138F0803198D282C
:10008000F03091000E0880389000F0309103031991
:10009000910003198F0303198D284E286120030155
:1000A0000C1820088E1F20088E0803190301900FDA
:1000B0005B28800642285C280000452884178005BC
:1000C0008D280D080C0403198C0A80300C1A8D063B
:1000D0000C198D068C188D060D0D8C0D8D0D8D282F
:1000E0008D01E83E8C008D09FC30031C7A288C07BA
:1000F000031877288C0764008D0F77280C18802848
:100100008C1C842800008428080003108D0C8C0CA3
:10011000FF3E031885280C088D28831303138312D0
:1001200064000800831603308500013086008312C6
:100130000612831606128312061383160613831201
:1001400086128316861283128610831686108312F7
:100150000611831606118312861183168611053047
:100160008312A2000830A00073308E000A303720BE
:1001700032308E000A3037200630A2000130A00055
:1001800004309F0001205A3C031DC2280120A40016
:1001900064002408413C031DCE280F21640024087C
:1001A000423C031DD428312164002408433C031D34
:1001B000DA28202164002408443C031DE028422161
:1001C00064002408453C031DF1280530A2000830D6
:1001D000A00073308E000A30372032308E000A3093
:1001E000372064002408463C031D0E29061283169E
:1001F00006128312061383160613831286128316C1
:1002000086128312861083168610831206118316B7
:10021000061183128611831686118312BC280616D6
:10022000831606128312061783160613831286148A
:100230008316861083120615831606118312080092
:1002400006168316061283120617831606138312E8
:1002500086148316861083128615831686118312E0
:100260000800061683160612831286168316861257
:1002700083128614831686108312861583168611C0
:10028000831208000616831606128312861683163A
:10029000861283128614831686108312061583161F
:0A02A00006118312080063005329C1
:02400E00F53F7C
:00000001FF
